:10000000830103308A00002B8C0003088301C200A7
:100010000408C3003C08C6003D08C7003E08C800ED
:100020003F08C9004008CA004108CB000B1D192831
:100030001A28EC2A0B119308031D1F282028832857
:100040002808B5022A089807051A2C282728960898
:10005000031D2C282B282E282D283028A801A80A7B
:100060008312051E392834289608031D392838289C
:100070003B283A283E28A8011830B5008312051EF7
:10008000472842289608031947284628492848281F
:100090004D28AA01AA0A9701970A17308312BD00BA
:1000A0001D0864239400051A5B2856289708031935
:1000B0005B285A285D285C286828AA01A8019801B5
:1000C0009301930A9201920A0F30B600F030B70004
:1000D000B508031D71286C289608031D7128702827
:1000E0007328722883281830B5008312051A7E28D9
:1000F00079289608031D7E287D2880287F2883285C
:100100009601960AA801930803198C2887289E084F
:10011000031D8C288B288E288D285429980A0C3092
:100120008312BE000030BF001D08BC00BD0170235B
:100130001730C0070318C10A1808BC00BD014108E8
:10014000803ABE003D08803A3E02031DA9283C08C3
:1001500040020318AC28AD28C2280230240203183C
:10016000B228B328BA28A801AA01980192019601E1
:100170009701930102302402031CBF28C028C22823
:100180009E019E0A92080319CB28C6288312051ED9
:10019000CB28CA28CD28CC28D12818089900980146
:1001A00092019208031DDA28D5288312051ADA284D
:1001B000D928DC28DB28542918089A0098019201D4
:1001C000920A9D08031DE528E6280C291A088312C7
:1001D000BC00BD011908BE00BF010130BE070318F5
:1001E000BF0A3F08803AC0003D08803A4002031D24
:1001F000FB283C083E02031CFE28FF280C29013086
:100200008312BC002508BD00BD0A08290310BC0DDF
:10021000BD0B06293C088F009D08031910291129E0
:10022000372919088312BC00BD011A08BE00BF019E
:100230000730BE070318BF0A3F08803AC0003D08D8
:10024000803A4002031D26293C083E02031C29294E
:100250002A29372901308312BC002508BD00BD0AB8
:1002600033290310BC0DBD0B31293C088F00240835
:100270002B3E840000080F078312BC0024082B3E8D
:1002800084003C088000A50A2508083A031D492976
:100290004A295429A5012408043A031D502951294B
:1002A00053299E019E0AA40A8E08031D5D29582920
:1002B0009E0803195D295C295E2963299008031DA6
:1002C0006329622965296429A82900308312051948
:1002D0000130013CBC003C083C07BC0000308519E3
:1002E0000130013C3C07BC00BC0EF030BC053C08B2
:1002F0008D00A601A0297D297D29831688188129D2
:1003000082297C290D0826078312890026082B3EA6
:1003100084000008880003108B1F8F2990299129E1
:1003200003148B138316081555308900AA308900F1
:1003300088140811031C9D299E299F298B17A60A42
:1003400005302602031CA529A6297B299001900AC5
:100350008E08031DB129AC2990080319B129B029D1
:10036000B329B229B7290F30B6000F30B7008E0875
:100370000319C029BB299E080319C029BF29C22916
:10038000C129222A9001900AA8010F2A8F01A601F3
:10039000DA29280EF03926078312890083160814FB
:1003A000831208089F0026082B3E840000081F06C1
:1003B0008F07A60A05302602031CDF29E029C92978
:1003C0008F08031DE429E5290E2AA808031DE92941
:1003D000EA29ED291508013C95002803031DF129A0
:1003E000F229F92903303002031CF729F829F929E9
:1003F000B0032808023A031DFE29FF29062A3230DD
:1004000030020318042A052A062AB00A2808033AEB
:10041000031D0B2A0C2A0E2A9C019C0AA80A0430F0
:100420002802031C142A152AC629A6011C2A2608FC
:100430002B3E84008001A60A05302602031C212AD7
:10044000222A172A8E0803192B2A262A9008031914
:100450002B2A2A2A2D2A2C2A3A2AAA01A8019001FD
:1004600096019701930198019E019201A401A501B3
:100470001830B5009508031D432A3E2A8E0803193B
:10048000432A422A452A442A492AFF30B600FF302F
:10049000B700950803194D2A4E2AEC2AB403B40874
:1004A000031D532A542AB02A31088312BE00BF010B
:1004B0001108BE02031CBF032708BC00BD013F0892
:1004C0003D06031D652A3E083C06031D682A692A6D
:1004D0008F2AB808031D6D2A6E2A702A0330B800CF
:1004E000B8033808023A031D762A772A7B2A320895
:1004F0009B00230891003803031D7F2A802A842A49
:1005000020089B0021089100B808031D882A892A29
:100510008D2A22089B00330891001B0AA700380887
:10052000023A031D942A952A9A2AB901BA01BA0AF5
:10053000BB01BB0A3803031D9E2A9F2AA42AB901C6
:10054000B90ABA01BB01BB0AB808031DA82AA92A27
:10055000AE2AB901B90ABA01BA0ABB013108B4001E
:1005600034082706031DB52AB62ADE2AA903A908DE
:10057000031DBB2ABC2ABF2A3008A900A70A3808D5
:10058000023A031DC42AC52ACA2AB901B90ABA0106
:10059000BB01BB0A3803031DCE2ACF2AD42AB901D6
:1005A000B90ABA01BA0ABB01B808031DD82AD92A68
:1005B000DE2AB901BA01BA0ABB01BB0A0F308312A5
:1005C000BD0039086423F03EB6000F30BD003A0E7E
:1005D000F0393B076423B70083124608BC00470884
:1005E000BD004808BE004908BF004A08C0004B08CB
:1005F000C10043088400420883008C0E0C0E0900E1
:100600000D3084003030122383010330C500F430F4
:10061000C400303084003C3016238301852B04064F
:100620008001840A0406031900340F2BBC00202328
:100630008000840A04083C0603190034172BC40008
:10064000C51B292B45088A004408C40A0319C50A9A
:1006500082008313451883174408C40A84000008E5
:02066000080090
:1006BC00360885003708860083120800BC0000301D
:1006CC003D183C070310BC0D0310BD0CBD080319ED
:1006DC000800662BC001C1010310BF0CBE0C031C2B
:1006EC007E2B3C08C0073D0803183D0AC1070310C8
:1006FC00BC0DBD0D3E083F0403190034722BFF30B6
:10070C00831685008601D0308100831281010B1184
:10071C008B168B17A601972B26082B3E8400800185
:10072C00A60A05302602031C9C2B9D2B922B32080B
:10073C009B00230891001B0AA7003008A900003079
:10074C008312851901308E008519AD2BAE2BD72B5A
:10075C00003005190130013C01399D00B62BB62B38
:10076C0083168818BA2BBB2BB52B0F30831289003C
:10077C001D08880003108B1FC42BC52BC62B03141C
:10078C008B138316081555308900AA3089008814FC
:10079C000811031CD22BD32BD42B8B17FF308316B1
:1007AC0085008E080319DB2BDC2BE12BF030831634
:1007BC0085009501950A0F30831289008316081461
:1007CC00831208089D00F22B9C08031DEE2BEF2BC7
:1007DC00F02B640083125E23EA2B002B0A34403486
:1007EC000134013401341834FF34FF340234013441
:0407FC00013401348F
:02400E00F6FFBB
:00000001FF
